:020000040000FA
:20040000FFCFFECFFDCFFCCFFBCFFACFF9CFF8CFF7CFF6CFF5CFF4CFF3CFF2CFF1CFF0CF74
:20042000EFCFEECFEDCFECCFEBCFEACFE9CFE8CFE7CFE6CFE5CFE4CFE3CFE2CFE1CFE0CF54
:20044000DFCFDECFDDCFDCCFDBCFDACFD9CFD8CFD7CFD6CFD5CFD4CFD3CFD2CFD1CFD0CF34
:20046000CFCFCECFCDCFCCCFCBCFCACFC9CFC8CFC7CFC6CFC5CFC4CFC3CFC2CFC1CFC0CF14
:20048000BFCFBECFBDCFBCCFBBCFBACFB9CFB8CFB7CFB6CFB5CFB4CFB3CFB2CFB1CFB0CFF4
:2004A000AFCFAECFADCFACCFABCFAACFA9CFA8CFA7CFA6CFA5CFA4CFA3CFA2CFA1CFA0CFD4
:2004C0009FCF9ECF9DCF9CCF9BCF9ACF99CF98CF97CF96CF95CF94CF93CF92CF91CF90CFB4
:2004E0008FCF8ECF8DCF8CCF8BCF8ACF89CF88CF87CF86CF85CF84CF83CF82CF81CF80CF94
:200500007FCF7ECF7DCF7CCF7BCF7ACF79CF78CF77CF76CF75CF74CF73CF72CF71CF70CF73
:200520006FCF6ECF6DCF6CCF6BCF6ACF69CF68CF67CF66CF65CF64CF63CF62CF61CF60CF53
:150540005FCF5ECF5DCF5CCF5BCF5ACF59CF58CF57CF56CF55B2
:200AAB00FFCFFECFFDCFFCCFFBCFFACFF9CFF8CFF7CFF6CFF5CFF4CFF3CFF2CFF1CFF0CFC3
:200ACB00EFCFEECFEDCFECCFEBCFEACFE9CFE8CFE7CFE6CFE5CFE4CFE3CFE2CFE1CFE0CFA3
:200AEB00DFCFDECFDDCFDCCFDBCFDACFD9CFD8CFD7CFD6CFD5CFD4CFD3CFD2CFD1CFD0CF83
:200B0B00CFCFCECFCDCFCCCFCBCFCACFC9CFC8CFC7CFC6CFC5CFC4CFC3CFC2CFC1CFC0CF62
:200B2B00BFCFBECFBDCFBCCFBBCFBACFB9CFB8CFB7CFB6CFB5CFB4CFB3CFB2CFB1CFB0CF42
:200B4B00AFCFAECFADCFACCFABCFAACFA9CFA8CFA7CFA6CFA5CFA4CFA3CFA2CFA1CFA0CF22
:200B6B009FCF9ECF9DCF9CCF9BCF9ACF99CF98CF97CF96CF95CF94CF93CF92CF91CF90CF02
:200B8B008FCF8ECF8DCF8CCF8BCF8ACF89CF88CF87CF86CF85CF84CF83CF82CF81CF80CFE2
:200BAB007FCF7ECF7DCF7CCF7BCF7ACF79CF78CF77CF76CF75CF74CF73CF72CF71CF70CFC2
:200BCB006FCF6ECF6DCF6CCF6BCF6ACF69CF68CF67CF66CF65CF64CF63CF62CF61CF60CFA2
:130BEB005FCF5ECF5DCF5CCF5BCF5ACF59CF58CF57CF5627
:010BFF00CF26
:00000001FF
